:0200000480007A
:1000000093000000130100009301000013020000A0
:100010009302000013030000930300001304000088
:100020009304000013050000930500001306000070
:100030009306000013070000930700001308000058
:10004000930800001309000093090000130A000040
:10005000930A0000130B0000930B0000130C000028
:10006000930C0000130D0000930D0000130E000010
:10007000930E0000130F0000930F0000B7E2010081
:1000800073A00230930210009392F20163CA02003F
:10009000130510009712000023A6A2F66FF05FFF71
:1000A00097020000938242047390523097410000FF
:1000B0009381C179178200001302B2F8137202FC17
:1000C000732540F1930510006370B500130115000E
:1000D0001311110133014100131615013302C2003F
:1000E0006F20904C130101EF2322110023242100E3
:1000F0002326310023284100232A5100232C6100AC
:10010000232E710023208102232291022324A102A5
:100110002326B1022328C102232AD102232CE10283
:10012000232EF1022320010523221105232421057A
:100130002326310523284105232A5105232C610557
:10014000232E710523208107232291072324A10751
:100150002326B1072328C107232AD107232CE1072F
:10016000232EF10773252034F325103413060100E4
:10017000EF20C02D73101534B72200009382028047
:1001800073A0023083204100032181008321C1003C
:100190000322010183224101032381018323C10141
:1001A0000324010283244102032581028325C10225
:1001B0000326010383264103032781038327C10309
:1001C0000328010483284104032981048329C104ED
:1001D000032A0105832A4105032B8105832BC105D1
:1001E000032C0106832C4106032D8106832DC106B5
:1001F000032E0107832E4107032F8107832FC10799
:0802000013010111730020300D
:1010000000000000000000000000000000000000E0
:1010100000000000000000000000000000000000D0
:1010200000000000000000000000000000000000C0
:1010300000000000000000000000000000000000B0
:081040000000000000000000A8
:10200000130101FEB7F3FFFF232E1100232C8100E3
:10201000232A910023282101232631012324410171
:1020200023225101B30375003717000063F2E33830
:10203000974F0000938F0FFDB38FAF00B384F5016E
:10204000138A050013DF2F0093D42400F327003AEE
:10205000B706FFFF9386F60FB3F7D7007390073AE2
:1020600073100F3B7390143B13070790B3E7E7001F
:102070007390073A73000012B302B500637A550CEF
:1020800017430000130343F837E4FDFFB7150200C0
:10209000131F2F00939424003303A300938E030097
:1020A00093880F009306050013084000B71900003D
:1020B000172E0000130E8EF91304F47F938505800C
:1020C00013092000130710009307F7FFB3F7D70099
:1020D0006392070663FE3E2D63E6E80B63F4980AFD
:1020E0006374E80E6362E30F6370930E930740001E
:1020F000138647003336E6002320CE00F327003056
:10210000B3F78700B3E7B7006308270B6308070935
:10211000F3970730038006007390073083270E0083
:1021200063980708131717009307F7FFB3F7D70053
:10213000E38207FA13171700E378E8F8938646005E
:1021400093884800938E4E0013034300E3EC56F649
:102150009307FAFF33674501B3F7E700638A070681
:102160008320C1010324810183244101032901014A
:102170008329C100032A8100832A4100130101023F
:102180006780000013060000E378E8F6E366E3F7F3
:10219000E37493F6138647006FF0DFF5F39707308B
:1021A00003A006007390073083270E00E38807F82A
:1021B00013052000EF00501AF39707300390060034
:1021C000739007306FF09FF5130640006FF09FF299
:1021D0009307400063E64713B71700009387071083
:1021E000130E100193581A009388F8FFB388F80172
:1021F00093D828007327003AB706FFFF9386F60F9F
:102200003377D7007310073A7350003B7390183B35
:10221000B3E7E7007390073A73000012E37255F4D6
:1022200017480000130848DE37EFFDFFB71E020015
:102230003308A80093054000137E8E011309800126
:10224000B714000017230000130343E0130FFF7FB0
:10225000938E0E801304200093091000938AF9FFD7
:10226000B3FAAA00639E0A0693870800930610003B
:1022700063062E0FB386F6009396260093972700E9
:1022800063F8931263E6FF0863F0DF0A63FE35111B
:10229000636CF810637AD810930A400093874A0061
:1022A000B3B737012320F300F3270030B3F7E7017A
:1022B000B3E7D701638C8908638CB90CF3970730B7
:1022C000030005007390073083270300E39207EEB5
:1022D00093991900938AF9FFB3FAAA00E3860AF8E2
:1022E00093991900E3FC35F713054500938F4F00D0
:1022F0009383430013084800E36055F66FF05FE6F0
:10230000B727000093870790130E90016FF09FEDA1
:1023100063F235036360F80293070000E374D8F8B2
:1023200093874A006FF0DFF763F635016364F800C6
:10233000E366D8F6930700002320F300F32700306C
:10234000B3F7E701B3E7D701E39889F6F3970730CE
:1023500003100500739007306FF01FF7130600029B
:1023600093062000130710006F00C001134AF7FF07
:102370001306F6FFB3F747019396160013171700DD
:10238000E30A06EE337AF700E3120AFE6FF09FEEDF
:10239000F39707300320050073900730832703006D
:1023A000E38407F46FF0DFE0930740006FF05FEF26
:1023B00013053000EF00407A130101FE2324410190
:1023C000232E1100130A0502232C8100232A9100D9
:1023D0002328210123263101232251011305450021
:1023E000930710006364AA0093078000B309F040CC
:1023F000939929009389090293040002930A3000FB
:1024000033099A401304400063FC9A0093050400CA
:102410001305090013044400EFF09FBEE3F884FEA7
:102420009384C4FFE39E34FD8320C1010324810112
:1024300083244101032901018329C100032A81006A
:10244000832A41001301010267800000130101FF8C
:1024500023261100930720006304F504972700004A
:1024600083A7C7BE6382070493075000631EF5026B
:1024700083D705008320C10017270000232807BC4D
:1024800093F73700B337F000B307F04093F7270016
:10249000938727003385F500130101016780000051
:1024A00013050000EF00406B13051000EF00C06A39
:1024B000130101EB23229113B70C00409387FCFF1B
:1024C000232481142322911423202115232A51131C
:1024D00023261114232E3113232C41132328611397
:1024E00023267113232481132320A113232EB1113A
:1024F0001309050093840500130406002324D1006A
:10250000930A50022326F1006F0040016304050680
:102510009385040013041400E70009000345040038
:10252000E31655FF83461400930D140013870D0026
:10253000930B00029309F0FF130AF0FF93050000CC
:1025400013065005130590009387D6FD93F7F70FF8
:1025500013041700636CF60617280000130888841C
:1025600093972700B387070183A70700B387070165
:10257000678007008320C11403248114832441143D
:10258000032901148329C113032A8113832A4113C8
:10259000032B0113832BC112032C8112832C4112B4
:1025A000032D0112832DC111130101156780000055
:1025B000938B0600834617001307040013041700CB
:1025C0009387D6FD93F7F70FE378F6F89385040029
:1025D00013055002E700090013840D006FF01FF48B
:1025E00003481700938906FD13070400930708FDAD
:1025F000930608006366F50293972900B3893701B3
:102600001307170093991900B389090103480700BC
:10261000938909FD930708FD93060800E37EF5FC06
:10262000E3540AF2138A09009309F0FF6FF0DFF117
:1026300083461700130704006FF01FF19385040011
:1026400013055002E70009006FF05FED832781005A
:10265000834617001307040083A9070093874700E8
:102660002324F1006FF0DFFB1305000393850400C2
:10267000E70009009385040013058007E7000900BF
:1026800083278100130C00012322010013874700D8
:1026900083278100930D000083A907002324E10014
:1026A00013060C00930600001385090093850D00A6
:1026B000EF10001C2328A10093070000930C0500D5
:1026C0006380B723130B4101130D100013060C0098
:1026D000930600001385090093850D00EF00105646
:1026E00013060C009306000093090500938D050066
:1026F000EF100018832741002320AB002320A10105
:10270000930C0500130B4B00130D1D00E390B7FD58
:10271000E3FE89FB635C4D01130AFAFF9385040015
:1027200013850B00E7000900E3484DFF83270100F4
:102730000327C10093099000338AE700131A2A0087
:1027400093070101338A47016F00C000832C0A0000
:10275000130ACAFFB3B79901B307F04093F77702A2
:10276000938707033385970193850400E7000900E9
:102770009307C100E39C47FD6FF05FDA93071000F9
:1027800063CCB716032781009307470063860518BB
:10279000832907002324F10013DCF941634E0C1850
:1027A000930D0C0023220100130CA0006FF05FEFCB
:1027B000130C0001232201009307100063C2B7101D
:1027C00083278100138747006FF09FEC83278100E8
:1027D00083AD0700138B470063840D1863584009CD
:1027E0009307D002639EFB0403C50D006308050236
:1027F000930BF0FF63C609009389F9FF638E79019B
:1028000093850400938D1D00E700090003C50D00AA
:10281000130AFAFFE31005FE635C4001130AFAFF96
:102820009385040013050002E7000900E3180AFE7F
:10283000232461016FF09FCE971D0000938D8D5270
:1028400093870D00B3863D01639809006F00401324
:10285000938717006386D70003C70700E31A07FEB4
:10286000B387B741330AFA40634C401103C50D00EA
:10287000E30005FC930BF0FF6FF0DFF79347FAFFDF
:1028800093D7F74183461700337AFA001307040001
:102890006FF09FCB832781009385040003A5070079
:1028A000138B4700E7000900232461016FF01FC765
:1028B0008346170093851500130704006FF0DFC8E7
:1028C00083278100138B7700137B8BFF93078B008B
:1028D00083290B00832D4B002324F1006FF05FDC74
:1028E000E3F289DF9307100023200100130D10008D
:1028F000E3C447E36FF09FE383278100138B7700E6
:10290000137B8BFF93078B0083290B00032C4B0059
:102910002324F1006FF09FE8032781006FF05FE749
:10292000130C8000232201006FF01FE9130CA0009C
:10293000232201006FF05FE8938504001305D002A5
:10294000E700090033373001B3078041B309304154
:10295000B38DE740130CA000232201006FF05FD479
:10296000635640019307D002E398FBEC971D0000EB
:10297000938D4D3F13058002930BF0FF6FF09FE79F
:10298000130AFAFF9385040013850B00E700090082
:10299000E30E0AEC130AFAFF9385040013850B007B
:1029A000E7000900E31E0AFC6FF05FEC83A7050057
:1029B0002380A70083A705009387170023A0F500B5
:1029C00067800000130101F81308F103137808FC75
:1029D000130700042320E800930700002322F800D7
:1029E000130710002324E800930700002326F800B3
:1029F0002328A800232AB800232CC800232ED8009F
:102A00000F00F00F97E6FFFF9386C65F23A0060135
:102A10009307000023A2F60097E6FFFF93868662E5
:102A200003A7060083A746003367F700E30A07FE03
:102A30001307000023A0E6009307000023A2F6007E
:102A40000F00F00F0325080083254800130101083B
:102A500067800000130101FF232481008325020405
:102A60009307020023261100B387B70013861500D1
:102A70002380A7002320C2049307A0006300F5026F
:102A800093070004630CF6008320C1000324810037
:102A90001305000013010101678000009356F64101
:102AA0001305020093050000EFF0DFF18320C10061
:102AB00023200204032481001305000013010101F7
:102AC00067800000732700B0971700009387C758EE
:102AD000631E050083A607001716000013060629CB
:102AE0009715000023A6C5563307D74023A0E7005B
:102AF000732720B0631E050083A647001716000049
:102B0000130646279715000023A6C5543307D74060
:102B100023A2E700678000009316150013E7160054
:102B200097E6FFFF9386064E9307000023A0E6007A
:102B300023A2F6006F0000003716000097E7FFFFA2
:102B40009387474C130636A79306000023A0C700BF
:102B500023A2D7006F000000130101FF23261100FC
:102B6000EFF09FFB97E7FFFF9387C7491306D0104D
:102B70009306000023A0C70023A2D7006F00000027
:102B8000834705006382070213060500834716008A
:102B900013061600E39C07FE3306A64093060000CA
:102BA000930500006FF01FE213060000930600007B
:102BB000930500006FF01FE16310050067800000BF
:102BC000130101FD13070500232611021305C1009F
:102BD0001306B101130890006F00800013860700F0
:102BE0009377F700B337F800B307F04093F7770215
:102BF0009376F70093870703B387F6002300F60068
:102C00009396C501135747009307F6FF33E7E60095
:102C100093D54500E314C5FC230E0100EFF05FF6E9
:102C20008320C1021301010367800000130101FC2E
:102C300013034102130E05002322B1022324C10213
:102C40002326D10217050000130505E193060300B2
:102C500013060E0093050000232E11002328E10225
:102C6000232AF102232C0103232E110323266100C2
:102C7000EFF01F848320C10113050000130101043C
:102C800067800000130101FB1303810323248102E9
:102C90002326A100232CC102232ED10213040500F8
:102CA0001386050017050000130585D09305C100A4
:102CB00093060300232611022322F1042320E104BA
:102CC0002324010523261105232E6100EFF04FFE7A
:102CD0008327C100238007000325C1008320C10290
:102CE000330585400324810213010105678000003C
:102CF000B3E7C500B367F50093F73700B306C50027
:102D0000638407023386C50093070500637ED502FE
:102D100003C705009385150093871700A38FE7FE6F
:102D2000E318B6FE67800000E37ED5FE930705003A
:102D300003A70500938747009385450023AEE7FE70
:102D4000E3E8D7FE6780000067800000B367C50036
:102D500093F737003306C5006380070293F5F50F3C
:102D6000930705006370C50493871700A38FB7FE10
:102D7000E31CF6FE6780000093F5F50F13978500BE
:102D800033E7E500931707013367F700E374C5FEE7
:102D9000930705009387470023AEE7FEE3ECC7FEE9
:102DA0006780000067800000130101F6975700005C
:102DB0009387472523244109175A0000130A8A24C0
:102DC00023263109B309FA40232A9108232821092F
:102DD000930405001389050013050200938507007D
:102DE00013860900232E1108232C81082322510960
:102DF000930A0200EFF0DFEF175600001306C62417
:102E0000330646419305000033853A01EFF01FF485
:102E10009305090013850400EFF01FDA9305000005
:102E200013050000EF00D065171900001309C9222F
:102E3000832609001304F103137404FC93040500B2
:102E400063940604832649006396060013850400F4
:102E5000EFF09FCC13090400971900009389491FD4
:102E600003A6490013050900971500009385C5F2D4
:102E7000EFF05FE13309A900E30A24FD1305040024
:102E8000EFF01FD06FF09FFC971900009389491C49
:102E900003A6090097150000938505F013050400AB
:102EA000EFF05FDE832649003309A400E38606FCC9
:102EB0006FF01FFB83470500638E07009307050033
:102EC00003C7170093871700E31C07FE3385A7404D
:102ED00067800000130500006780000013060500EE
:102EE000B306B60013850500930706006398050036
:102EF0006F00C001938717006388F60003C70700BF
:102F0000E31A07FE3385C740678000006780000032
:102F100083470500938515001305150003C7F5FFCA
:102F200063880700E386E7FE3385E740678000009B
:102F3000930700006FF05FFF9307050003C70500CC
:102F40009387170093851500A38FE7FEE31807FE0C
:102F50006780000003470500930600029307050001
:102F60006318D70003C7170093871700E30CD7FE39
:102F70009306D0026300D7069306B0026300D7041D
:102F800083C6070093050000638206041305000052
:102F900093871700138606FD1317250083C60700C5
:102FA0003305A700131515003305A600E39206FEAE
:102FB000638005023305A0406780000083C61700C8
:102FC0009305000093871700E39206FC13050000A9
:102FD0006780000083C617009305100093871700D1
:102FE000E39606FA130500006FF09FFE138F0500AD
:102FF0001308000063DC0500B337A000B305B04040
:10300000338FF5403305A0401308F0FF63DA060064
:10301000B335C0003307D040B306B7403306C040D5
:1030200093080600138706009307050093050F0019
:1030300063940624B7460080938686EF6376CF0EAE
:10304000370301006378660C1303F00F6374C30049
:10305000130780003353E600B386660003CE0600F4
:10306000330EEE00130700023303C741630CC701A0
:10307000B3156F00335EC501B3186600B365BE00BB
:10308000B317650013D60801B3F6C50213950801FE
:103090001355050113D70701B3D5C5029396060151
:1030A00033E7E600B305B502637AB70033071701CB
:1030B000636617016374B700330717013307B7401E
:1030C000B376C7029397070193D707013357C70217
:1030D0003307E50213950601B367F50063FAE700CD
:1030E000B387170163E6170163F4E700B38717019D
:1030F000B387E74033D5670093050000630A0800F3
:10310000B337A000B306B040B385F6403305A04006
:10311000678000003703000113070001E36C66F2CB
:10312000130780016FF01FF3631606009308100069
:10313000B3D8E8023706010063F6C8121306F00F91
:10314000637416011307800033D6E800B386C60007
:1031500003CE0600B3051F41330EEE001307000235
:103160003303C7416306C709B3986800B35ECF0154
:10317000B3176500335EC50113D50801B3156F00A1
:10318000336EBE009395080193D5050113560E01C9
:10319000B3D6AE0233F7AE02B386D50213170701DA
:1031A0003367C700637AD7003307170163661701D7
:1031B0006374D700330717013306D7403377A6026D
:1031C000131E0E01135E0E013356A60213170701DC
:1031D0003386C502B365C70163FAC500B38515011F
:1031E00063E6150163F4C500B3851501B385C540D9
:1031F00093D6080133F7D50213950801135505013D
:1032000013D60701B3D5D502131707013367C700DB
:10321000B305B502637AB700330717016366170178
:103220006374B70033071701B305B74033F7D5020E
:103230009397070193D70701B3D5D502B305B5021C
:1032400013150701B367F50063FAB700B3871701D9
:1032500063E6170163F4B700B3871701B387B7407C
:103260006FF05FE93706000113070001E3EEC8ECD9
:10327000130780016FF05FEDE362DFE837070100BD
:1032800063FAE604930EF00F33B7DE00131737002E
:10329000B748008033D3E600938888EFB38868008E
:1032A00083CE0800B38EEE0013070002330ED74121
:1032B000631CD70363E4E601636AC500B307C54036
:1032C000B305DF403335F500B385A540138507000E
:1032D0006FF0DFE2B708000113070001E3EA16FB15
:1032E000130780016FF0DFFA3357D601B396C6019A
:1032F000B36FD700B357DF0113D70F0133F3E702E2
:10330000B315CF01B356D501B3E6B60093950F01BF
:1033100093D5050193D806013316C6013315C501AF
:10332000B3D7E70213130301B3681301338FF50218
:103330001383070063FEE801B388F8011383F7FFE6
:1033400063E8F80163F6E8011383E7FFB388F80147
:10335000B388E84133FFE8029396060193D606014D
:10336000B3D8E802131F0F01336FDF00B3851503D5
:1033700093870800637EBF00330FFF019387F8FF38
:103380006368FF016376BF009387E8FF330FFF0197
:10339000B305BF4013130301370F01003363F3007C
:1033A0009307FFFFB378F30093560601135303010D
:1033B000B377F6003387F802B307F302B388D80275
:1033C0003303D302B388F80093560701B38616017E
:1033D00063F4F6003303E30193D7060133836700F8
:1033E000B70701009387F7FFB3F6F600939606013F
:1033F0003377F7003387E60063E66500639E650078
:10340000637CE5003306C7403337C7003307F70155
:103410003303E340130706003307E5403335E50087
:10342000B3856540B385A540B397D5013357C70130
:1034300033E5E700B3D5C5016FF05FCC9308050015
:103440009387050013080600138506001383080000
:1034500063940628B7460080938686EF63F6C50E10
:10346000370701006378E60C1307F00F3337C70006
:10347000131737003355E600B386A60083C606004F
:10348000130500023387E600B306E540630CE50050
:10349000B397D70033D7E8003318D600B365F700E9
:1034A0003393D80093580801B3D7150313160801B6
:1034B0001356060113570301B3F6150313850700CE
:1034C000B305F6029396060133E7E600637EB70084
:1034D000330707011385F7FF636807016376B700B9
:1034E0001385E7FF330707013307B740B3771703A7
:1034F0001313030113530301335717039397070162
:1035000033E36700B306E60213060700637CD300CB
:10351000330368001306F7FF636603016374D30087
:103520001306E7FF131505013365C5009305000079
:103530006F00400E3705000113070001E36CA6F28F
:10354000130780016FF01FF36316060013071000C6
:103550003358C702370701006370E80C1307F00FF8
:1035600063740701130580003357A800B386E60093
:1035700003C70600130600023307A700B306E640A0
:103580006316E60AB38707419305100093580801B4
:10359000131608011356060113570301B3F6170358
:1035A000B3D717039396060133E7E600330EF6020E
:1035B00013850700637EC701330707011385F7FFF3
:1035C000636807016376C7011385E7FF33070701C7
:1035D0003307C741B37717031313030113530301D1
:1035E000335717039397070133E36700B306E602E7
:1035F00013060700637CD300330368001306F7FF4C
:10360000636603016374D3001306E7FF1315050116
:103610003365C5006780000037070001130500010E
:10362000E364E8F4130580016FF01FF43318D80049
:10363000B3D5E7003393D800B397D70033D7E8006A
:10364000935808013366F70033F715039317080101
:1036500093D7070113550601B3D5150313170701B7
:103660003367A700B386B70213850500637ED700D2
:10367000330707011385F5FF636807016376D700F9
:103680001385E5FF33070701B306D74033F7160369
:103690001316060113560601B3D6160313170701B6
:1036A000B388D702B367C7001387060063FE17010C
:1036B000B38707011387F6FF63E8070163F6170175
:1036C0001387E6FFB387070193150501B3871741F9
:1036D000B3E5E5006FF09FEB63E6D518370701000F
:1036E00063F4E6041307F00FB335D7009395350064
:1036F0003747008033D5B600130787EF3307A7009D
:1037000003470700130500023307B700B305E54080
:103710006316E50213051000E3EEF6EE33B5C800BC
:10372000134515006FF01FEF3707000193050001E7
:10373000E3E0E6FC930580016FF09FFB3353E60066
:10374000B396B6003363D30013550301B31EB6001E
:1037500033D6E700B376A602B397B70033D7E800B5
:103760003368F7009317030193D707011357080134
:103770003356A6029396060133E7E600338FC7025D
:10378000130E0600637EE70133076700130EF6FF92
:10379000636867006376E701130EE6FF330767008F
:1037A0003307E741B376A7023357A7029396060182
:1037B0003386E7029317080193D70701B3E7F600B2
:1037C0009306070063FEC700B38767009306F7FF01
:1037D00063E8670063F6C7009306E7FFB3876700F7
:1037E00013150E01370E01003365D5009306FEFF59
:1037F0003378D500B387C740B3F6DE001356050112
:1038000093DE0E013303D802B306D6021357030129
:103810003308D8033308D800330707013306D6032B
:103820006374D7003306C601935607013386C6007A
:1038300063E6C702E39CC7CEB70701009387F7FF93
:103840003377F700131707013373F300B398B80009
:103850003307670093050000E3FEE8DA1305F5FF80
:103860006FF0DFCC93050000130500006FF09FDAC6
:1038700093080600138706009307050013880500C8
:10388000639C0622B7460080938686EF63FCC50CD6
:1038900037030100637E660A1303F00F6374C300ED
:1038A000130780003353E600B386660003CE06009C
:1038B000330EEE00130700023303C741630CC70148
:1038C000B3956500335EC501B31866003368BE006A
:1038D000B317650013D608013377C80213950801A2
:1038E0001355050193D607013358C8021317070172
:1038F000B366D7003308050363FA0601B3861601E1
:1039000063E6160163F40601B3861601B386064129
:1039100033F7C6029397070193D70701B3D6C602C0
:10392000B306D50213150701B367F50063FAD70094
:10393000B387170163E6170163F4D700B387170154
:10394000B387D74033D56700930500006780000038
:103950003703000113070001E36666F413078001D3
:103960006FF05FF46316060013061000B3581603D9
:103970003706010063F2C80A1306F00F63741601DC
:103980001307800033D6E800B386C60003CE0600D6
:10399000330EEE00130700023303C7416318C70953
:1039A000B385154113D70801139508011355050177
:1039B00013D60701B3F6E502B3D5E50293960601E7
:1039C000B3E6C600B305B50263FAB600B3861601C6
:1039D00063E6160163F4B600B3861601B385B640FC
:1039E000B3F6E5029397070193D70701B3D5E50234
:1039F000B305B50213950601B367F50063FAB70086
:103A0000B387170163E6170163F4B700B3871701A3
:103A1000B387B7406FF01FF33706000113070001AB
:103A2000E3E2C8F6130780016FF0DFF5B398680092
:103A300033D7C501B3176500335EC50113D508013F
:103A4000B376A702B3956500336EBE009395080167
:103A500093D5050113560E013357A702939606011D
:103A6000B3E6C6003387E50263FAE600B3861601C3
:103A700063E6160163F4E600B38616013386E6407A
:103A8000B376A602131E0E01135E0E013356A60274
:103A9000939606013386C502B3E5C60163FAC500F5
:103AA000B385150163E6150163F4C500B3851501FF
:103AB000B385C5406FF01FEFE3EAD5E83707010093
:103AC00063FCE604130EF00F3337DE0013173700E4
:103AD000B748008033D3E600938888EFB388680046
:103AE00003CE0800330EEE00130700023303C74174
:103AF000631EC70363E4B600636AC500B307C5402D
:103B0000B385D5403335F5003388A54013850700CC
:103B1000930508006FF09FE3B70800011307000149
:103B2000E3E816FB130780016FF09FFA3357C601D5
:103B3000B3966600336FD700B3D7C50113570F0193
:103B4000B3F8E702B39565003358C5013368B80090
:103B500093150F0193D5050193560801331666009E
:103B600033156500B3D7E70293980801B3E6D80090
:103B7000B38EF5029388070063FED601B386E60193
:103B80009388F7FF63E8E60163F6D6019388E7FFC1
:103B9000B386E601B386D641B3FEE60213180801E8
:103BA00013580801B3D6E602939E0E01B3EE0E0140
:103BB000B385D5029387060063FEBE00B38EEE0187
:103BC0009387F6FF63E8EE0163F6BE009387E6FF96
:103BD000B38EEE01B385BE4093980801B70E010085
:103BE000B3E8F8009387FEFF33F8F8009356060118
:103BF00093D80801B377F6003307F802B387F802C9
:103C00003308D802B388D8023308F8009356070166
:103C1000B386060163F4F600B388D801B707010044
:103C20009387F7FF13D80601B3F6F60093960601C3
:103C30003377F700B30818013387E60063E6150110
:103C4000639E1501637CE5003306C7403337C70028
:103C50003307E701B388E840130706003307E54060
:103C60003335E500B3851541B385A540B397C5014C
:103C70003357670033E5E700B3D565006FF01FCD1C
:103C8000973700009387073817160000130686370A
:103C900093D7C700130101FF1357C6009397A700DE
:103CA0002326110023248100232291009725000060
:103CB0009385453593E7770C1317A7001367170013
:103CC00093D6C5002322F600B707008023A0E500A5
:103CD000B3E7F600739007189307F0FF7390273B44
:103CE000B70719007390073A37150000EFE0CFECE3
:103CF000B7240000138504FEEFE00FECB7150000B9
:103D000037150000EFE0CFAF3714000093050480B3
:103D100037150000EFE0CFAE1385048093050480D3
:103D2000EFE00FAE8320C100032481008324410013
:103D3000130500001301010167800000130101FF5A
:103D4000170500001305C50323261100EFE05FE30C
:103D50008320C1001305F0FF1301010167800000FB
:103D6000286E756C6C2900006D6379636C650000CA
:103D70006D696E737472657400000000496D706C3B
:103D8000656D656E74206D61696E28292C20666FE3
:0D3D90006F210A002573203D2025640A00E4
:103DA00090E8FFFF2CE8FFFF9CE8FFFF2CE8FFFFF7
:103DB0002CE8FFFF2CE8FFFF2CE8FFFFACE8FFFF3B
:103DC0002CE8FFFF2CE8FFFF10E8FFFFDCEAFFFF15
:103DD0002CE8FFFF10E8FFFF40E8FFFF40E8FFFF8F
:103DE00040E8FFFF40E8FFFF40E8FFFF40E8FFFF3B
:103DF00040E8FFFF40E8FFFF40E8FFFF2CE8FFFF3F
:103E00002CE8FFFF2CE8FFFF2CE8FFFF2CE8FFFF6A
:103E10002CE8FFFF2CE8FFFF2CE8FFFF2CE8FFFF5A
:103E20002CE8FFFF2CE8FFFF2CE8FFFF2CE8FFFF4A
:103E30002CE8FFFF2CE8FFFF2CE8FFFF2CE8FFFF3A
:103E40002CE8FFFF2CE8FFFF2CE8FFFF2CE8FFFF2A
:103E50002CE8FFFF2CE8FFFF2CE8FFFF2CE8FFFF1A
:103E60002CE8FFFF2CE8FFFF2CE8FFFF2CE8FFFF0A
:103E70002CE8FFFF2CE8FFFF2CE8FFFF2CE8FFFFFA
:103E80002CE8FFFF2CE8FFFF2CE8FFFF2CE8FFFFEA
:103E90002CE8FFFF2CE8FFFF2CE8FFFF2CE8FFFFDA
:103EA000F4EAFFFFDCE9FFFF2CE8FFFF2CE8FFFF4F
:103EB0002CE8FFFF2CE8FFFF2CE8FFFF2CE8FFFFBA
:103EC0002CE8FFFF10EBFFFF2CE8FFFF2CE8FFFFC3
:103ED00080EBFFFFC8E8FFFF2CE8FFFF2CE8FFFFA7
:103EE0002CEAFFFF2CE8FFFF8CEBFFFF2CE8FFFF25
:103EF0002CE8FFFF10EAFFFF0001020203030303A7
:103F00000404040404040404050505050505050569
:103F10000505050505050505060606060606060649
:103F20000606060606060606060606060606060631
:103F30000606060606060606070707070707070719
:103F40000707070707070707070707070707070701
:103F500007070707070707070707070707070707F1
:103F600007070707070707070707070707070707E1
:103F700007070707070707070808080808080808C9
:103F800008080808080808080808080808080808B1
:103F900008080808080808080808080808080808A1
:103FA0000808080808080808080808080808080891
:103FB0000808080808080808080808080808080881
:103FC0000808080808080808080808080808080871
:103FD0000808080808080808080808080808080861
:103FE0000808080808080808080808080808080851
:083FF000080808080808080889
:103FF8001000000000000000037A5200017C01015B
:104008001B0D02001000000018000000D8EFFFFF91
:104018005004000000000000100000002C00000008
:1040280014F4FFFF3404000000000000100000003A
:104038004000000034F8FFFF1004000000000000FA
:040000058000000077
:00000001FF
